:0200000480007A
:100000009710000093800000171100001301810277
:1000100083A1000013F2110093F2F17F13F3F1FFBB
:1000200093F3010013F401802320310023224100C7
:10003000232451002326610023287100232A8100F4
:1000400097100000938040FC17110000130101007D
:1000500003A40000937414001375F47F9375F4FFE8
:1000600013760400937604802320810023229100DC
:100070002324A1002326B1002328C100232AD10074
:1000800097100000938080F817110000130181FD84
:1000900083A6000013F7160093F7F67F13F8F6FF18
:1000A00093F8060013F906802320D1002322E100F3
:1000B0002324F1002326010123281101232A2101F1
:1000C000971000009380C0F417110000130101FB8A
:1000D00003A9000093791900137AF97F937AF9FF45
:1000E000137B0900937B0980232021012322310106
:1000F000232441012326510123286101232A710170
:1001000097100000938000F117110000130181F88F
:1001100083AB000013FC1B0093FCFB7F13FDFBFF74
:1001200093FD0B0013FE0B8023207101232281011C
:10013000232491012326A1012328B101232AC101EF
:10014000171D0000130D4DED971D0000938D0DF64A
:10015000032E0D00937EFE0713FFFE03937FFF0126
:1001600093F0FF0013F170009371310023A0CD01D3
:1001700023A2DD0123A4ED0123A6FD0123A81D0078
:1001800023AA2D0023AC3D0097100000938000E9C6
:1001900017110000130141F383A2000013F01200B5
:1001A0002320010097100000938080E717110000C2
:1001B0001301C1F183A2000013F01200937210002A
:1001C000232001002322510097100000938080E536
:1001D00017110000130101F083A1000013F2F1FFD9
:1001E0009372F2FF13F3F2FF1377F3FF9377F7FFA6
:1001F00013F8F7FF937CF8FF13FDFCFF937DFDFFE1
:1002000023203100232241002324A1012326B10110
:1002100017150000130505E297150000938585EC7E
:10022000370610F01306C6F26306B5028326C50032
:100230002320D600832685002320D6008326450070
:100240002320D600832605002320D60013050501B0
:100250006FF09FFD370510F0130505F22320050010
:04026000000000009A
:101000000000000001000000FFFFFFFFFFFFFF7F67
:1010100000000080FFFFCDAB7856341298BADCFE9A
:10102000145892360000000000000000000000008C
:10103000FFFFFFFFFFFFFFFFFFFFFFFFFFFFFFFFC0
:10104000FFFFFFFFFFFFFFFFFFFFFFFFFFFFFFFFB0
:10105000FFFFFFFFFFFFFFFFFFFFFFFFFFFFFFFFA0
:10106000FFFFFFFFFFFFFFFFFFFFFFFFFFFFFFFF90
:10107000FFFFFFFFFFFFFFFFFFFFFFFFFFFFFFFF80
:10108000FFFFFFFFFFFFFFFFFFFFFFFFFFFFFFFF70
:10109000FFFFFFFFFFFFFFFFFFFFFFFFFFFFFFFF60
:1010A000FFFFFFFFFFFFFFFFFFFFFFFFFFFFFFFF50
:1010B000FFFFFFFFFFFFFFFFFFFFFFFFFFFFFFFF40
:1010C000FFFFFFFFFFFFFFFFFFFFFFFFFFFFFFFF30
:1010D000FFFFFFFFFFFFFFFFFFFFFFFFFFFFFFFF20
:040000058000000077
:00000001FF
